:020000040000FA
:10000000340A440831084D0831082E083108200808
:1000100062087908200841084C0842082E08200888
:1000200061086C0862084008630872086F08770866
:1000300064082E0872087508200828084308290853
:10004000430852084F08570844082008520875080A
:1000500073087308690861082C0820083208300802
:040060003008330829
:040064000008000888
:080068002500850C0200390C93
:100070000600B40C2800320C290067006C006D00EB
:100080006E00FF0C2F0007040607480A07056705E6
:1000900006023B008A012B001B022A008B071E0B65
:1000A00061004704780C92000307620AB3027307E9
:1000B0007C0A74007300C7067C0AC705960C3500DD
:1000C00076007C0AB40294077C0A73007400C707A8
:1000D0007C0AC704160243077A0AA7070707720AB1
:1000E0000704790AA7046C006D006E00960C2800C6
:1000F00007057C0A080CA7017200C707990AF503D7
:10010000F600B602160235074306990A07068A0A60
:10011000070567046707930AA902780C8900780C21
:1001200003062900990AE9000A0C89000A0C030752
:1001300029008705960C8800030687040902070733
:100140009B0CA706110288004306AA0AFF0C0307AE
:10015000010CE801A707B30AF003F100B102F107AF
:10016000B30AA7040704CF06CB0AAF02CF07CB0A16
:10017000E7041A024306BF0A080CA701CB0AA70727
:100180000707C40A0704CB0AA7046C006D006E00C1
:10019000960C28000705E707EA0AF903FA00BA02F5
:1001A0001A024306EA0A0706D70A07056704030C82
:1001B00059014307EA0A6707E40AA902780C890093
:1001C000780C03062900EA0AE9000A0C89000A0CE7
:1001D00003072900EC03EF0AED03EE00AE02360C34
:1001E0008E000307F70A6C006D006E00070408021A
:1001F000810003071A0B47061C0B8706660047059C
:100200002705F703F800B8021807070B78006B07FB
:10021000480A04006A07170BDC0C97000307170B4A
:100220006F00E706170BE705640C39007A007700CA
:100230007800480A00000000010B230B27071D0B64
:0E024000FF0C26002704A606B2020400F70AEF
:021FFE00EE0FE4
:00000001FF
